:100000000C94E1020C9419030C9419030C94190339
:100010000C9419030C9419030C9419030C941903F0
:100020000C9419030C9419030C9440100C947C0F3D
:100030000C94641B0C9419030C9419030C9419036D
:100040000C9419030C9419030C9419030C941903C0
:100050000C9419030C9417110C9419030C941903A4
:100060000C9419030C9419030C9419030C941903A0
:100070000C9419030C9419030C9419030C94190390
:100080000C9419030C9419030C9419030C94751C0B
:100090000C9419030C9419030C9419030C94190370
:1000A0000C9419030C9419030C941903BD04CF0488
:1000B000DD04EE04070511053505DA07DA070E0839
:1000C0000E087A08A50A340AA50A9C087A098D093F
:1000D0008D09410A6E0A490A4C0A550A4F0A580A04
:1000E000950DBC0D540FBC0D540F040E270E540F6C
:1000F000160F290F0004010402040304040405047C
:1001000000050105020503050405050500060106B5
:100110000206030604060506000701070207030797
:1001200004070507000001000200030004000500A9
:1001300000010101020103010401050100020102A5
:100140000202030204020502000301030203030387
:100150000403050305010980A101850319012AB7DC
:1001600000150126B700950175108100C0050C0926
:1001700001A101850419012AA002150126A00295FA
:100180000175108100C005010906A101050719E0EC
:1001900029E715002501950875018102950175086B
:1001A00081010507190029FF150026FF0095067536
:1001B0000881000508190129059505750191029529
:1001C0000175039101C009023B00020100A0320940
:1001D0000400000103010100092111010001224076
:1001E0000007058103080001090401000103000064
:1001F00000092111010001223200070582032000BD
:10020000011201000200000008DEC03713100201D5
:100210000200010A03480075006D00610000001C27
:10022000034B0067004F00660048006500640067EC
:1002300000650068006F0067007300000004030998
:1002400004350014000800150017000A00E000043F
:10025000001A00070009000500E300E2001600068E
:100260000019002C62000000001D001B002B452817
:10027000442F0013000C0018001C000B00347133D5
:100280000012000E000D001100307831740F00369E
:100290000010002A7200000000380037004C452989
:1002A0004435003400370013001C000C00E000044B
:1002B000003600080018001B00E300E20012000DE9
:1002C000000E002C6200000000330014002B4528B3
:1002D000442F000F0006000A0009000700387116BD
:1002E00000150017000B0005003078317411001A5A
:1002F0000010002A72000000001D0019004C452962
:100300004435001400090013000A000700E000044F
:10031000001A00160017000500E300E200150006B1
:100320000019002C62000000001D001B002B452856
:10033000442F00330018000F000D000B0034711221
:10034000001C00080011000E00307831740C0036DB
:100350000010002A7200000000380037004C4529C8
:10036000443500140015001A0005000A00E00004DE
:100370000007000B0017001900E300E20016001050
:100380000006002C62000000001D001B002B452809
:10039000442F003300180009000D001C0034710CBC
:1003A000001300080011000E00307831741200367E
:1003B000000F002A7200000000380037004C452969
:1003C000442D023A003C003D003E0022022E611EF8
:1003D000023B00200221022200010057641F02207C
:1003E0000021000100000000001E001F00010001AC
:1003F0000044004300410040003F0023022D7127CC
:10040000024200250224022300457801002602252D
:100410000024000100000000002700260001000168
:10042000005300540060006100560057002E6155D3
:10043000005F005D005E008500010001005C005A65
:10044000005B000100000000006200590001000193
:10045000003900470046004A00A900A8006571491C
:10046000004B0052005000AA00010001004F005153
:10047000004D0001000000000048004E0001000196
:1004800000015C000000000000000000000000AA65
:100490005D0000A85DA75D0000005C0753A95D003A
:1004A000000000F056000000000000000001000104
:1004B00000015C000000000000000000000000AA35
:1004C0005D0000A85DA75D0000005C0753A95D000A
:1004D000000000F0560000000000000000010001D4
:1004E0000000000000CA5CC75CC65CC85C0000007D
:1004F00000BF5CCB5CC95CC45C00000753BE5CC33E
:100500005CC55C010000000000C25CC05C01000131
:100510000000000000CA5CC75CC65CC85C0000004C
:1005200000BF5CCB5CC95CC45C00000753BE5CC30D
:100530005CC55C010000000000C25CC05C01000101
:1005400000000000000000000000000001010203A4
:10055000040506080A0C0F1114181C2024292E3338
:10056000393F464C535B626A7179818A929AA2AA9A
:10057000B2B9C1C8CFD5DCE1E7EBF0F4F7FAFCFD86
:10058000FEFFFEFDFCFAF7F4F0EBE7E1DCD5CFC8A7
:10059000C1B9B2AAA29A928A8179716A625B534CFC
:1005A000463F39332E2924201C1814110F0C0A0839
:1005B0000605040302010100000000000000000025
:1005C000000011241FBECFEFDAE0DEBFCDBF04B6BE
:1005D00003FE18C080911A0290911B02A0911C0288
:1005E000B0911D028730904BA740B04B59F4109248
:1005F0001A0210921B0210921C0210921D02E0E0DF
:10060000F8E3099511E0A0E0B1E0EAE4FCE302C000
:1006100005900D92AE34B107D9F722E0AEE4B1E017
:1006200001C01D92AA31B207E1F70E943C170C9459
:10063000231E0C940000CF92DF92EF92FF92C12C08
:10064000D12C7601C39404C0CC0CDD1CEE1CFF1C25
:100650008A95D2F76C2D83E090E00E947C1DC70143
:10066000B601FF90EF90DF90CF900C94081AEF92B4
:10067000FF920F931F93CF93DF93CDB7DEB76797AA
:100680000FB6F894DEBF0FBECDBF4B8B5C8B6D8B6E
:100690007E8B8F8B242F0E891F8961111092C301CD
:1006A0000115110531F05F3F31F481E02F3F19F45E
:1006B00003C081E001C080E080FD37C0A22FB0E020
:1006C00081E090E07C01022E01C0EE0C0A94EAF772
:1006D000852F90E0662319F03091810105C0FC015F
:1006E000E05BFE4F30813E213323C1F046E0489F5E
:1006F0009001499F300D11242A0F3B1F220F331FF9
:10070000F901EB50FF4F5491F901EC50FF4F249148
:10071000FC01E05BFE4F9081E92A06C0FC01E05B32
:10072000FE4FE0948081E822E08286E0FE013D9663
:10073000DF01982F1D929A95E9F72D875E876F87C5
:10074000198B088BDE01179601900D928A95E1F7BF
:10075000CE0107960E948D1581113EC086E0FE01F4
:100760003796DE01119601900D928A95E1F7FF818F
:10077000E8856A857B856115710531F0EF3F31F4BD
:1007800081E0FF3F19F403C081E001C080E080FDFB
:1007900023C02091880130E0C90101968770992714
:1007A0004091B90150E08417950779F1F983EA8304
:1007B0007D836C8396E0929FD001939FB00D1124AE
:1007C000A757BE4FFE01319601900D929A95E1F721
:1007D000809388010E94FB1416E08091B9019091EA
:1007E00088018917F9F0189FC001112487579E4F7F
:1007F0000E948D158823B1F08091B90190E0019697
:10080000877099278093B901E8CF0E94321A10921D
:1008100088011092B901E2E8F1E086E0DF011D9263
:100820008A95E9F767960FB6F894DEBF0FBECDBF85
:10083000DF91CF911F910F91FF90EF90089581FB71
:10084000992790F980FD02C02E9A01C02E9891112F
:1008500002C02D9A08952D9808954F925F926F923D
:100860007F928F929F92AF92BF92CF92DF92EF9240
:10087000FF920F931F93CF93DF93CDB7DEB72A97E5
:100880000FB6F894DEBF0FBECDBFFC010081D18052
:1008900083819481892B41F044244A94D41006C06A
:1008A00091E00F3F19F403C091E001C090E090FD8A
:1008B000CAC67F0185E0DE01169601900D928A95E9
:1008C000E1F7F70122818E819F81222349F00E9466
:1008D000F218182F682F8E819F810E94781903C00B
:1008E0000E944B19182F20E3129FF001112486E07B
:1008F000D89EE00DF11D1124E00FF11DEE0FFF1F3A
:10090000EF5BFD4F05911491F7018281083AFDE5F7
:100910001F07A1F028F4073A9DE5190751F01FC001
:10092000093AEDE51E0789F00A3AFDE51F0791F047
:1009300016C0882309F460C680E004C0882309F447
:100940005BC681E00E941B0357C6882309F454C686
:1009500082E0F8CF882309F44FC683E0F3CF8823E1
:1009600009F4AAC0F801EC5BFC45E730F10508F09A
:10097000A3C0EA5AFF4F0C94F61D80910C028770B9
:10098000886280930C02887F91E009F490E0809166
:100990000C0290FB80F980930C0285E007C08091E7
:1009A0000C0287708E7F80930C0280E00E94E81C0E
:1009B00080910C020E94161D1FC680910C02982F78
:1009C00096959695969509F45EC0915E990F990F4C
:1009D000990F8770892B80930C023AC020910C02EA
:1009E000822F869586958695482F50E04530510593
:1009F00054F48F5F982F990F990F990F822F87705A
:100A0000892B80930C0280910C02816029C0809117
:100A10000C0280FF03C00E941B1DEEC50E94281D12
:100A2000EBC580910C02282F2695269526952F5FE1
:100A30002F71922F990F990F990F8770892B80939F
:100A40000C02263018F0877080930C0280910C0203
:100A5000887F91E009F490E080910C0290FB80F98E
:100A600080930C020E94161D0EC080910C0281FF23
:100A700012C08D7F80930C020E94161D8091710020
:100A80008E7F8093710080910C0286958695869565
:100A90000E94E81CB1C5826080930C020E94161D62
:100AA00010920F0210920E0210920D0280917100AE
:100AB000816080937100A0C5043F9CE5190799F4FB
:100AC00006E221EE40EE64EF7CE509C0083D9CE5BE
:100AD000190711F506E221EE41EE68ED7CE5C7014C
:100AE0000E94DF1B89C5053FECE51E0708F05CC1CD
:100AF000093DFCE51F0731F407E225EE45EE69EDFF
:100B00007CE5EDCF0A3D2CE5120701F708E221E074
:100B100045EE6AED7CE5E3CF882309F47AC11092B3
:100B2000120204302DE5120758F40B3F8CE518072C
:100B300080F4C80182509C45449708F054C109C014
:100B400002369DE5190729F0063AEDE51E0709F082
:100B50004AC10E94FC139093DA018093D9010131BC
:100B6000FCE51F0709F4C6C008F042C009308CE557
:100B7000180709F49BC000F50530ECE51E0709F4E1
:100B800085C078F403302CE5120709F478C008F02A
:100B90007AC002301C4509F0F7C08091D90181600C
:100BA000F1C00730ECE51E0709F478C008F07AC000
:100BB0008091D9018061E6C00D302CE5120709F45F
:100BC00087C058F40B309CE5190709F479C008F088
:100BD0007BC08091D90188606FC00F30FCE51F0792
:100BE00009F480C008F082C08091D901877FCAC013
:100BF0000E3F8CE5180709F471C000F50531ECE5EE
:100C00001E0709F485C068F403312CE5120709F4C6
:100C100075C008F095C00E94321A8091D9018F7773
:100C2000B1C00C3F9CE51907A9F108F054C00B3F77
:100C30001C4509F0A9C08091DA0140C002302DE5C1
:100C4000120709F489C058F401159DE5190709F444
:100C50005AC008F069C08091DA0182602FC0023664
:100C6000FDE51F0709F47EC0063A2DE5120709F4D9
:100C700083C003301D4509F087C060E06EC08091DD
:100C8000D90182607FC08091D90116C08091D901BD
:100C9000886078C08091DA0182604FC08091D9016C
:100CA000806270C08091D90180646CC00E94321A49
:100CB0008091D901806866C0846064C081603DC055
:100CC0008091D9018E7F5EC08091D9018D7F5AC0FD
:100CD0008091D90116C08091DA0118C08091DA01A3
:100CE0008D7F2BC08091D9018F7E4CC08091D9011E
:100CF0008F7D48C08091D9018F7B44C08091D901FC
:100D0000877F8B7F3FC08091DA018D7F8E7F15C0FA
:100D10008091D90182FB222720F991E0922790FB54
:100D200082F990FB83F92EC08091DA01982F90957B
:100D300091708E7F892B90FB81F98093DA0124C01A
:100D40000E94321A8091D90187FB222720F991E075
:100D5000922790FB87F916C061E08EE090E00E9438
:100D60007C1D12C08091D90184FB222720F991E0DB
:100D7000922790FB84F906C08091D901982F909515
:100D800090FB80F98093D9016091D9011091DA012B
:100D900084E090E00E947C1D612F82E290E00E943E
:100DA0007C1D0E94321A28C4063FECE51E0731F470
:100DB00006E221EE42EE66EF7CE591CE063FFCE5D1
:100DC0001F0730F407E225EE44EE65EF7CE587CEA1
:100DD000073F2CE5120709F09FCE07E225EE46EE0D
:100DE00067EF7CE57CCE06318CE5180759F58091DC
:100DF000C4018A7A91E009F490E090935801882325
:100E000011F065E301C069E288E791E00E948D1B63
:100E100016C006311C4509F06BC08091580188232B
:100E200009F40FC485E3E8E7F1E02EE731E09281B1
:100E3000891301C0128231962E173F07C1F70E9415
:100E40008514DAC30B359DE5190709F44CC058F435
:100E50000115FCE51F07C1F00F3D1C4509F048C016
:100E60000E940D14C9C30C358DE5180709F43DC067
:100E70000D351D4509F03CC08091DA0182FB8827C1
:100E800080F991E0892732C00E94321AEFEFF4E333
:100E90002CE0E150F0402040E1F700C0000081E08C
:100EA0008093E00080E28093D8001092C9008FE127
:100EB0009EE40197F1F700C0000087E090EBDC01B1
:100EC00080931A0290931B02A0931C02B0931D0200
:100ED0009CE088E10FB6F894A895809360000FBE5F
:100EE00090936000FFCF81E001C080E00E94DE149B
:100EF000F70182810081D180882359F0802F9D2DB8
:100F00000E94F218182F682F802F9D2D0E947819AB
:100F100005C0802F9D2D0E944B19182F20E3129F92
:100F2000F001112486E0D89EE00DF11D1124E00FA0
:100F3000F11DEE0FFF1FEF5BFD4F859194910E9415
:100F40006B12082FD92EB82EF7011281858082945A
:100F5000BFE08B228091BA018770E1F01123D1F0BC
:100F6000892F807F803449F090E2900F983090F084
:100F7000803619F4F6EF0F1769F08091DA0182FDDF
:100F800009C082E00E94C1148091BA018770AA242E
:100F9000A3948111A12C9D2C9294FFE09F22892D76
:100FA00090E08C30910508F0D0C2FC01E35AFF4F6D
:100FB0000C94F61D9D2D9F708D2D807FC92E19F0EC
:100FC000C294E0EFCE221123B9F0CC2009F438C24C
:100FD00080E2800F883010F0B11006C08091C4010B
:100FE000C82AC092C40105C08091C301C82AC0921A
:100FF000C3010E94851424C2802F0E944E1ACC2067
:1010000009F4A3C2005E083098F1BB2089F1C094B6
:101010008091C301C822C092C3012DC09D2D9F7035
:101020008D2D807FC92E803219F0C29470EFC722B7
:10103000BB2029F044244394B414E9F14CC08091BE
:10104000DA0182FF1BC0112369F0CC2039F08091B6
:10105000C401C82AC092C4010E94851480E00E9485
:101060007F1A73C280E00E944E1ACC2009F46DC230
:101070008C2D0E947E140E94851467C2112389F072
:101080008091C501882059F055245394851007C0DC
:10109000C82AC81609F459C2C092C50156C28C2983
:1010A00012C0882029F066246394861409F44DC286
:1010B0000E9478141BC0112349F065E0762E781445
:1010C00008F443C28C2D0E94441A3FC224E0281524
:1010D00008F43BC20BC0112319F0882099F3B0C16A
:1010E000882021F089E3B812BBC1B1C18C2D0E94C8
:1010F0003D1A2BC28D2D86958695837019F081300F
:1011000071F023C2112331F0802F9D2D93700E9426
:10111000BD1B23C280E090E00E94BD1B36C211239C
:1011200031F0802F9D2D93700E94A71B16C280E086
:1011300090E00E94A71B29C28D2D837009F069C021
:10114000111107C2902F929596959770990F990F4C
:10115000802F8F70482E512C612C712C092E04C0C9
:10116000440C551C661C771C0A94D2F704FF12C06D
:101170004FE050E060E070E004C0440F551F661F70
:10118000771F9A95D2F7DB01CA0180959095A095BB
:10119000B09503C080E090E0DC016D2D669566950A
:1011A0006370623019F1C8F42091C6013091C70113
:1011B0004091C8015091C901613059F084299529A5
:1011C000A629B729BC01CD0162237323842395236B
:1011D0000AC0422A532A642A752ABC01CD01642917
:1011E0007529862997290E94081AB3C1842995294F
:1011F000A629B7294090C6015090C7016090C80148
:101200007090C901BC01CD016425752586259725FF
:10121000EACF112319F08D2D817001C086958823A6
:1012200009F497C1902F929596959770990F990F01
:10123000802F8F70482E512C612C712C092E04C0E8
:10124000440C551C661C771C0A94D2F704FF12C08C
:101250004FE050E060E070E004C0440F551F661F8F
:10126000771F9A95D2F7DB01CA0180959095A095DA
:10127000B09503C080E090E0DC016D2D6695669529
:1012800063706230D9F068F52091D5013091D601B4
:101290004091D7015091D801613059F084299529A6
:1012A000A629B729BC01CD0162237323842395238A
:1012B0001EC0422A532A642A752A13C084299529FC
:1012C000A629B7294090D5015090D6016090D7014A
:1012D0007090D801BC01CD01642575258625972520
:1012E00006C0BC01CD0164297529862997290E9471
:1012F000A4192FC12D2D2F70C22E112339F0822F4A
:101300000E94E719802F0E94441A23C1802F0E9457
:101310003D1A8C2D0E94C2191CC1802F92EFB91664
:1013200009F449C09B1538F0E0EFBE1671F0F1EFFB
:10133000BF16E1F180C053EF452EB41409F442C04A
:1013400044EF542EB51471F176C0112329F134E025
:10135000632E681408F4F9C02D2D2F7181E090E000
:10136000A0E0B0E0AC01BD0104C0440F551F661FF2
:10137000771F2A95D2F78091D5019091D601A0913F
:10138000D701B091D8012A013B01482659266A2687
:101390007B26C301B2012BC025E0522E581408F45D
:1013A000D4C0DACF8091DA0182FF24C0112329F062
:1013B0008D2D8F7132C01123D9F38D2D8F710E9425
:1013C000C219C3C0112381F02D2D2F7181E090E04F
:1013D000A0E0B0E0BC01CD0104C0660F771F881FFC
:1013E000991F2A95D2F703C060E070E0CB010E94FC
:1013F000A419ABC01123A1F00D2D0F71802F0E94F5
:10140000E7198091DA0182FD07C028E0029FC00140
:10141000112483608093BA01802F0E94E71995C040
:1014200081E00E94C11481E0881508F08EC082E03E
:101430000E94C1148AC0112329F0882009F4B8CF72
:10144000802F0DCE882009F4B8CF893349F49FEF5F
:10145000E7EEF3E09150E040F040E1F700C000001B
:10146000802F0E944E1A71C08B2D90E0FC01E05F2E
:10147000F109E730F10508F03FC0E759FF4F0C9440
:10148000F61D112309F481C09091810181E0892723
:1014900015C01093810161C081E081270FC0111137
:1014A0005CC081E08093810170C0111156C06BC097
:1014B000112339F082E08093590181E0809381010A
:1014C0004CC080915901823019F481E08093590118
:1014D00080915901833009F058C053C0112339F06D
:1014E00080918001882381F21092800136C094E0BF
:1014F000492E481448F649C0809180018820C1F0E7
:10150000882341F09091810181E0892780938101B6
:1015100010928001802F112319F00E947F1A1DC0A4
:101520000E944E1A86E0F70111928A95E9F72DC0C4
:10153000882399F0111111C09091810181E08927D0
:10154000809381011092800120C088EF890D843042
:1015500020F40E94D31B0E941F041123B1F08D2D93
:10156000807F803619F4F6EFBF1679F0809159012B
:10157000823019F483E080935901809159018130C0
:1015800021F41092590110928101AA20A9F08091B2
:10159000BA0180FD11C0F701128285958595859568
:1015A0000E94E719C7010E942D048091BA01859518
:1015B000859585950E94C21985E0F701DE01119697
:1015C00001900D928A95E1F789819A810E944B19C9
:1015D0009A8120E3829FF001112486E0989FE00D1C
:1015E000F11D11248981E80FF11DEE0FFF1FEF5B44
:1015F000FD4F8591949127C08091BA01877019F1B0
:10160000F70182818823F9F08091DA0182FD1BC005
:1016100082E02A960FB6F894DEBF0FBECDBFDF91F1
:10162000CF911F910F91FF90EF90DF90CF90BF90DF
:10163000AF909F908F907F906F905F904F900C94A1
:10164000C11489E2F0CB2A960FB6F894DEBF0FBE24
:10165000CDBFDF91CF911F910F91FF90EF90DF9061
:10166000CF90BF90AF909F908F907F906F905F9042
:101670004F9008952091E4003091E50095E6409167
:10168000EC00842F817040FF23C08091E80080FD32
:101690001DC080916E01882399F0853099F080916A
:1016A000EB0085FD11C04091E4005091E500241746
:1016B000350729F3915011F09A01E1CF84E00895A4
:1016C00082E0089583E0089581E0089580E0089520
:1016D0004091E80042FFDDCF0895EF92FF920F9313
:1016E0001F93CF93DF937C018B010E943A0B8111F2
:1016F00019C0E70101151105A1F08091E80085FDF1
:101700000AC08091E8008E778093E8000E943A0B2F
:10171000882381F307C089918093F100015011095A
:10172000E9CF80E0DF91CF911F910F91FF90EF9073
:1017300008958091700187FF11C08091E80082FDBB
:1017400005C080916E018111F8CF11C08091E80031
:101750008B770BC080916E01882349F08091E8005F
:1017600080FFF8CF8091E8008E778093E80008959D
:10177000982F973068F59093E900981739F0709199
:10178000EC002091ED005091F00003C0242F762F43
:1017900050E021FD02C09F5FECCF3091EB003E7F17
:1017A0003093EB003091ED003D7F3093ED003091B0
:1017B000EB0031603093EB007093EC002093ED0070
:1017C0005093F0002091EE0027FDE5CF80E00895D2
:1017D0008F708093E90081E0089520917601309127
:1017E00077012617370748F06115710539F4209104
:1017F000E8002E772093E80001C0B901FC0120E049
:101800006115710579F180916E018823F1F18530C0
:10181000F1F18091E80083FD3CC08091E80082FDF9
:101820002EC08091E80080FFEBCF2091F3008091E3
:10183000F20090E0922B6115710551F0883091050E
:1018400038F421912093F100615071090196F3CF92
:1018500021E0089709F020E08091E8008E778093DE
:10186000E800CECF2111CFCF0AC080916E0188232E
:1018700061F0853061F08091E80083FD0AC08091BD
:10188000E80082FFF2CF80E0089582E0089583E0CF
:10189000089581E008950895089580916301089561
:1018A00080935E017093600160935F0180916E018F
:1018B000843001F582E08093E9008FEF9091E80099
:1018C000815095FD06C095ED9A95F1F700008111C4
:1018D000F5CF8091E80085FF0DC040E050E063E067
:1018E00070E08EE591E00E946D0B8091E8008E77AC
:1018F0008093E8000895BC0184E00C94500CBC0176
:1019000083E00C94500CCF93DF9321E02093E90007
:101910002FEF3091E800215035FD06C035ED3A95A6
:10192000F1F700002111F5CF2091E80025FF14C048
:10193000EC0140E050E068E070E00E946D0B8091A7
:10194000E8008E778093E80088E0FE01A4E6B1E02D
:1019500001900D928A95E1F7DF91CF9108951F9341
:10196000CF93DF93CDB7DEB7AA970FB6F894DEBF5B
:101970000FBECDBFE0E7F1E088E791E02091F100F4
:1019800021938E179F07D1F780917101833009F45D
:1019900061C030F4813071F0823009F49BC0B2C074
:1019A0008A3009F487C08B3009F46CC0893009F0A3
:1019B000A9C020C080917001813A09F0A3C0809134
:1019C000E800877F8093E800809174019091750111
:1019D000892B21F468E084E691E003C060E080E0B8
:1019E00090E070E00E94ED0B8091E8008B7780938F
:1019F000E80088C080917001813209F083C0809135
:101A0000740190917501029708F07CC08091E80004
:101A1000877F8093E8008091E80082FD05C0809177
:101A20006E018111F8CF6EC02091F3008091F20019
:101A300090E0922B029731F48091F100813011F007
:101A4000863021F48091F100809363018091E80059
:101A50008B7754C080917001813A09F053C0809116
:101A6000740190917501892B09F04CC08091E800B8
:101A7000877F8093E8008091E80080FFFCCF809111
:101A8000000137C0809170018132E1F580917401CD
:101A900090917501892BB1F58091E800877F809343
:101AA000E8000E94990B80917201809300010E94CE
:101AB000321A28C080917001813221F58091E800AE
:101AC000877F8093E8000E94990B80917301809337
:101AD000620118C080917001813AA1F48091E80000
:101AE000877F8093E8008091E80080FFFCCF8091A1
:101AF00062018093F1008091E8008E778093E80086
:101B00000E94990B8091E80083FFCEC18091700103
:101B100090917101492F50E04A30510508F0C4C13D
:101B2000FA01E059FF4F0C94F61D803821F08238FD
:101B300009F0BAC108C080916C0190916D019923A0
:101B400089F082600FC0809174018F70873008F037
:101B5000ABC18093E9008091EB0085FB882780F979
:101B60001092E9009091E800977F9093E8008093AD
:101B7000F1001092F10065C1282F2D7F09F094C16A
:101B8000882319F0823061F08FC180917201813019
:101B900009F08AC1933009F080E080936D012EC076
:101BA0008091720181112AC0809174018F702FEF92
:101BB000280F263008F078C18093E9002091EB00CF
:101BC00020FF1CC0933021F48091EB00806214C090
:101BD0009091EB0090619093EB0021E030E0A9013F
:101BE00002C0440F551F8A95E2F74093EA00109215
:101BF000EA008091EB0088608093EB001092E9008E
:101C00008091E800877F20C181114EC1109172013F
:101C10001F778091E3008078812B8093E30080918F
:101C2000E800877F8093E8000E94990B8091E8008C
:101C300080FFFCCF8091E30080688093E300111166
:101C400002C082E001C083E080936E012DC1805804
:101C5000823008F029C180917201909173018C3D0E
:101C600053E0950779F583E08A838AE289834FB749
:101C7000F894DE01139620E03EE051E2E32FF0E01D
:101C800050935700E49120FF03C0E295EF703F5F4F
:101C9000EF708E2F90E0EA3010F0C79601C0C0962A
:101CA0008D939D932F5F243149F74FBF8091E800BA
:101CB000877F8093E8006AE270E0CE0101960E947F
:101CC000ED0BAEC04091740150917501292F33275F
:101CD00023303105A9F068F42130310509F4F3C04F
:101CE0002230310509F0E0C08BE390E0E6ECF1E052
:101CF00044C02132310521F12232310571F1D4C0C5
:101D0000992781309105A1F058F0029709F0CCC0D5
:101D1000E3E1F2E0E4918E2F90E0E3E1F2E02AC00B
:101D2000EDE3F2E0E4918E2F90E0EDE3F2E022C0EB
:101D3000EFE1F2E0E4918E2F90E0EFE1F2E01AC0E3
:101D40004115510509F4C4C04130510509F0ACC03A
:101D500089E090E0E1EFF1E010C04115510509F490
:101D6000BCC04130510509F09FC082E390E0E4E53A
:101D7000F1E003C0009709F497C02091E800277FA5
:101D80002093E80020917601309177018217930724
:101D900008F49C0140E02115310589F180916E0124
:101DA000882309F43DC08530D9F18091E80083FD96
:101DB00037C08091E80082FD2FC08091E80080FF4D
:101DC000EACF4091F3008091F20090E0942B21152E
:101DD000310559F08830910540F444914093F10069
:101DE0003196215031090196F2CF41E0089709F070
:101DF00040E08091E8008E778093E800CCCF4111DD
:101E0000CDCF0AC080916E01882351F0853041F01A
:101E10008091E80083FD04C08091E80082FFF2CF4A
:101E20008091E8008B778093E8003EC08038E1F530
:101E30008091E800877F8093E80080916F01809314
:101E4000F1008091E8008E778093E8000E94990B62
:101E50002BC0811129C08091720190917301992743
:101E6000029714F58091E800877F8093E800109135
:101E7000720110936F010E94990B111106C080919D
:101E8000E30087FD02C081E001C084E080936E0121
:101E900042E061EC81E00E94B80B42E261EC82E03A
:101EA0000E94B80B80916E018091E80083FF1AC0F8
:101EB0008091E800877F8093E8008091EB0080624A
:101EC0008093EB000FC082E190E0E1E0F2E055CFBB
:101ED00089E090E0E8EDF1E050CF80E490E0E6E8C2
:101EE000F1E04BCFAA960FB6F894DEBF0FBECDBF80
:101EF000DF91CF911F9108951F920F920FB60F920D
:101F000011242F933F934F935F936F937F938F93FE
:101F10009F93AF93BF93CF93DF93EF93FF93C091C2
:101F2000E900CF708091EC00D82FD17080FDD0E80F
:101F30001092E9008091F000877F8093F000789400
:101F40000E94AF0C1092E9008091F00088608093AD
:101F5000F000CD2BCF70C093E900FF91EF91DF919E
:101F6000CF91BF91AF919F918F917F916F915F9131
:101F70004F913F912F910F900FBE0F901F9018958A
:101F8000E8EDF0E080818E7F80831092E200109275
:101F9000DA001092E100A0EEB0E08C9181608C93A9
:101FA00080818F77808319BCA7EDB0E08C918E7F04
:101FB0008C9380818F7E8083109261010895CF92EF
:101FC000DF92EF92FF920F931F93CF93DF93C8EDB1
:101FD000D0E088818F7E8883E7EDF0E080818160AA
:101FE000808384E082BF81E08093610188818E7F5D
:101FF000888302EE10E0F80110821092DA0081EE80
:10200000C82ED12CF601108288818F778883888131
:102010008068888388818F7D888319BC10926E01C7
:1020200010926F0110926D0110926C0190EEE92EEA
:10203000F12CF70180818B7F808388818160888388
:1020400042E060E080E00E94B80BF60180818E7F64
:102050008083F801808181608083808188608083B3
:10206000F70180818E7F8083888180618883DF9102
:10207000CF911F910F91FF90EF90DF90CF90089537
:102080001F920F920FB60F9211242F933F934F93ED
:102090005F936F937F938F939F93AF93BF93EF93D0
:1020A000FF938091E10082FF09C08091E20082FFEE
:1020B00005C08091E1008B7F8093E1008091DA0080
:1020C00080FF2AC08091D80080FF26C08091DA006E
:1020D0008E7F8093DA008091D90080FF18C080E164
:1020E00089BD82E189BD09B400FEFDCF81E0809306
:1020F0006E018091610181110FC00E94C00F0E948A
:10210000DF0F8091E20084608093E20005C019BC7B
:1021100010926E01109261018091E10080FF17C062
:102120008091E20080FF13C08091E2008E7F809357
:10213000E2008091E20080618093E2008091D8000B
:1021400080628093D80019BC85E080936E018091F5
:10215000E10084FF30C08091E20084FF2CC080E168
:1021600089BD82E189BD09B400FEFDCF8091D80010
:102170008F7D8093D8008091E1008F7E8093E10075
:102180008091E2008F7E8093E2008091E200816086
:102190008093E20080916F01882311F084E007C0F2
:1021A0008091E30087FD02C081E001C083E080935D
:1021B0006E0180916E018091E10083FF27C08091C4
:1021C000E20083FF23C08091E100877F8093E100DC
:1021D00082E080936E0110926F018091E1008E7F0A
:1021E0008093E1008091E2008E7F8093E2008091F5
:1021F000E20080618093E20042E060E080E00E94C3
:10220000B80B8091F00088608093F000FF91EF910F
:10221000BF91AF919F918F917F916F915F914F91FE
:102220003F912F910F900FBE0F901F9018957894AB
:102230001F920F920FB60F9211248F939F93AF931B
:10224000BF9380915A0190915B01A0915C01B09184
:102250005D010196A11DB11D80935A0190935B0110
:10226000A0935C01B0935D01BF91AF919F918F915D
:102270000F900FBE0F901F9018952FB7F894809174
:102280005A0190915B01A0915C01B0915D012FBF5B
:10229000089580E008959091D90192FF0DC0282FF4
:1022A0002871283019F4877F846006C0282F247194
:1022B000243011F48B7F886093FF0DC0282F287184
:1022C000283119F4877E846106C0282F24712431B7
:1022D00011F48B7E88612091DA0120FF0DC0382F28
:1022E0003871383019F4877F816006C0382F31711A
:1022F000313011F48E7F886021FF0DC0282F2871A6
:10230000283119F4877E816106C0282F217121317F
:1023100011F48E7E886194FD877E0895F894E82FED
:10232000E295EF70F0E031A1282F2F7081E090E06E
:1023300001C0880F2A95EAF7982F9095932391A3CF
:1023400092A1892B82A3789408959F92AF92BF9215
:10235000CF92DF92EF92FF920F931F93CF93DF9371
:10236000CDB7DEB728970FB6F894DEBF0FBECDBF4E
:10237000AE014F5F5F4F7A0188E0FA0111928A95B2
:10238000E9F70FE311E06A01AA24A394B12CF80144
:1023900080818F3F09F441C0F894E82FE295EF70F7
:1023A000F0E021A18F70A50102C0440F551F8A954E
:1023B000E2F7CA01922F982B91A392A180958923CD
:1023C00082A3789400C0E7E4F1E0912C31E0219100
:1023D0002F3F89F0A22FA295AF70B0E090968C911C
:1023E00090E02F7002C0959587952A95E2F780FDC1
:1023F00002C0832F01C080E0982A330F51E0ED34F2
:10240000F50729F7F80180818F3F11F00E948E11A6
:10241000F0EAFA95F1F7F60190820F5F1F4FFFEF98
:10242000CF1ADF0A41E00734140709F0B0CF48E0C3
:1024300050E0B7018DEC91E00E94161E11E000976C
:1024400009F410E0892B89F088E0F701ADECB1E0E8
:1024500001900D928A95E1F781E08093CC010E9472
:102460003D119093CB018093CA018091CC018823C8
:10247000F9F02091CA013091CB014FB7F8948091C7
:102480005A0190915B01A0915C01B0915D014FBF39
:10249000821B930B059760F0EDECF1E0ACEDB1E041
:1024A00081918D9351E0E53DF507D1F71092CC0174
:1024B000812F28960FB6F894DEBF0FBECDBFDF91F7
:1024C000CF911F910F91FF90EF90DF90CF90BF9031
:1024D000AF909F900895CF93DF938238910569F173
:1024E000B0F48133910509F46FC048F48932910545
:1024F00009F465C08A32910509F46BC08AC085333E
:10250000910509F457C089339105B9F082C0833E23
:10251000910571F138F4803E9105B1F0823E91054C
:1025200011F177C0863E9105B9F1873E9105C9F159
:10253000843E910509F06DC024C02091D90120FD91
:1025400053C021FD51C065C08091D90180FD46C0B6
:102550008091DA0180FF48C08091D90184FD47C194
:1025600083EE90E046C18091D90182FF3AC0F4CF5A
:102570008091D90182FD35C08091DA0180FD34C09F
:10258000EBCF8091DA0181FF35C08091D90184FDC4
:102590002EC187EE90E02DC18091D90183FF27C025
:1025A000F4CF8091D90183FD22C08091DA0181FDB1
:1025B00021C0EBCF8091D90185FD1FC021C0809142
:1025C000D90185FD1DC019C08091D90186FD1BC0B0
:1025D0001DC08091D90186FD19C015C089E390E026
:1025E00008C182EE90E005C180EE90E002C186EE67
:1025F00090E0FFC084EE90E0FCC089E290E0F9C07A
:1026000085E390E0F6C08AE290E0F3C081E390E0D9
:10261000F0C0811532E5930708F069C0811541E5E6
:10262000940728F0982F8827816F906AE2C0883E2F
:10263000910568F5803E910508F0DBC0883A910568
:10264000B8F4853A910548F0855AE82FF0E0E25F4A
:10265000FE4F808190E09064CCC08130910509F4F8
:10266000C3C008F4C4C08430910508F4C0C0C1C020
:102670008F3B910508F0BBC0885AE82FF0E0EE0FC1
:10268000FF1FEF5EFE4F808191819464B2C081157F
:1026900020E59207F0F09C0174E0369527957A9535
:1026A000E1F7922F9370482F437021E030E002C091
:1026B000220F331F4A95E2F73C68392B8F70982F11
:1026C0009695969540E2949FC0011124822B932BFE
:1026D00090C0811530E4930718F09F70906A89C00C
:1026E0009C013A9521153F4108F483C080C0EC015C
:1026F000C11586E5D807E8F5C11525E5D20748F0EC
:102700008C2F0E944B118F7190E0982F8827906238
:1027100070C0C11534E5D30728F09C2F8827846F3B
:10272000906A67C0AE01437055272C2F26952695D9
:10273000C115D34578F481E090E002C0880F991F5D
:102740004A95E2F740E2249F90011124822B932BBB
:102750009C684FC081E090E002C0880F991F4A95A5
:10276000E2F740E2249F90011124822B932B9A6878
:1027700040C0C11529E5D20788F4C11538E5D30753
:1027800028F09C2F8827806F906A33C0C11547E5D9
:10279000D40768F5CE01992790662BC0C1158AE54C
:1027A000D80790F48C2F8F700E944B1194E0D6952F
:1027B000C7959A95E1F7CF70D0E0DC2FCC27D06990
:1027C0009E01282BC90115C0CE019056811590425B
:1027D00070F48D2F8F710E944B11282F2F71CE0115
:1027E00099279062922B05C081E090E002C080E0C2
:1027F00090E0DF91CF910895CF9384E090E00E9424
:102800006E1DC82F82E290E00E946E1D2C2F30E0DA
:10281000A901582BCA01CF91089569EE7EEF80E09F
:1028200090E00E949A1D60E082E090E00E947C1D92
:1028300060E083E090E00E947C1D1092C60110923F
:10284000C7011092C8011092C90160E084E090E0D5
:102850000E947C1D60E082E290E00E947C1D60E0AE
:1028600085E090E00E947C1D60E086E090E00E94A0
:102870007C1D6FEF87E090E00E947C1D40E050E0FF
:10288000BA0188E090E00E948E1D60E08DE090E04B
:102890000E947C1D40E050E0BA0188E190E00E9477
:1028A0008E1D60E087E190E00E947C1D40E050E0DA
:1028B000BA018CE190E00E948E1D60E070E080E241
:1028C00090E00E949A1D40E050E0BA0188E190E05B
:1028D0000E948E1D40E050E0BA018FE090E00E941F
:1028E0008E1D40E050E0BA0183E190E00C948E1D13
:1028F0008091C50181111092C50108958095909134
:10290000C40189238093C40108959091C4018091EA
:10291000C301982B909378018091C501882389F099
:10292000892B80937801EAE7F1E097E080E091500D
:1029300029F021912223D9F38F5FF9CF81110E94D1
:10294000781448E050E06BEB71E088E791E00E947A
:10295000161E892BA9F088E0E8E7F1E0ABEBB1E0C7
:1029600001900D928A95E1F7E0911502F09116021F
:10297000309731F00280F381E02D88E791E00994EF
:1029800008952091BA01809582238093BA01982FEF
:10299000977099F430E0482F082E000C550B24173F
:1029A000350759F09091DA0192FD07C0859585951C
:1029B00085950E94C2191092BA010895CF93C091D3
:1029C000DA01C2FB992790F9981799F080FBC2F9B8
:1029D000C093DA016091D90184E090E00E947C1DEF
:1029E0006C2F82E290E00E947C1D82E0CF910C94DB
:1029F000C114CF9108958091B901909188018917F0
:102A000019F08F5F8770FBCF08950F931F93CF93BB
:102A1000DF938091870182958F7009F05DC080916E
:102A20008401882309F458C08091B901109188016C
:102A30006091820170918301C0918501D0918601DE
:102A400091E06F3F09F090E0292F06E0811709F42B
:102A500043C0209721F07F3F21F030E003C031E0F8
:102A600001C0322F90E030FD34C0089FF001099F73
:102A7000F00D1124DF01A757BE4F11963C9111971D
:102A8000371327C03C91361324C012963C911297FD
:102A900031111FC013964D915C9114974C1B5D0B27
:102AA000483C5105B0F4809187018F70806180931C
:102AB0008701E257FE4F80818F708061808382E8BA
:102AC00091E00E942D04DF91CF911F910F910C9402
:102AD000FB1401968770BACFDF91CF911F910F91B0
:102AE0000895CF93DF93EC010E94F21820E3829FB8
:102AF000C0011124FC0126E0D29FE00DF11D11243C
:102B0000EC0FF11DEE0FFF1FEF5BFD4F85919491D0
:102B10000E946B12DF91CF9108959F92AF92BF9266
:102B2000CF92DF92EF92FF920F931F93CF93DF9399
:102B3000CDB7DEB761970FB6F894DEBF0FBECDBF3D
:102B40008C0185E0F801DE011D9601900D928A95B9
:102B5000E1F7F801E2809091820160918301409158
:102B60008501509186014115510531F06F3F31F4D7
:102B700081E09F3F19F403C081E001C080E0F82F9D
:102B8000F1709F2E80FD1AC1F80130812181C38030
:102B9000D48082E8A82E81E0B82EF0908401F6015E
:102BA000E41BF50BFF2009F4C6C080918701E83CC7
:102BB000F10508F091C0482F407F09F050C0621322
:102BC00011C093130FC0FE2CE1100CC08F708061F8
:102BD00080938701C5010E942D0480918701F8012F
:102BE000858337C1CD2831F02F3F31F481E03F3F5D
:102BF00019F403C081E001C080E080FD03C081E0E2
:102C00008E2502C080E090E0F82FF170FF2E80FF4B
:102C10001CC08091B9014091880156E0841709F4E5
:102C2000F6C090E0589FF001599FF00D1124E7572E
:102C3000FE4F6181261306C06081631303C0628169
:102C4000E61203C001968770E9CFFE2CEE2009F44E
:102C500000C18091870181608093870149C0621320
:102C600006C0931304C0E11002C0F80186C0C80179
:102C70000E94121A882351F1EE2041F12091870120
:102C8000822F82958F7090E0029774F0809182017C
:102C90009091830198878F831986DB86CA862C875B
:102CA000CE0107960E942D0486E0F801A2E8B1E06B
:102CB00001900D928A95E1F70E9405150AC06217EE
:102CC000C9F0C8010E94121A81111EC0C8010E94D9
:102CD0002D04FF24F394BDC0482F407F81F782E884
:102CE00091E00E942D0486E0F50111928A95E9F7A2
:102CF000F12CAFC09313E5CFE110E3CFF80185834A
:102D0000C8010E942D0454C0EE2001F320918701D8
:102D1000822F82958F7090E0029734F28091820129
:102D2000909183019A8389831B82DD82CC822E83DA
:102D3000CE010196B7CFE83CF105D0F5FE2CEE2090
:102D400029F2621327C0931325C02091870120FD2B
:102D500018C0822F82958F70482F50E04115510581
:102D600081F0F80125834F30510541F08F5F982F96
:102D70009295907F822F8F70892B8583C8010E9446
:102D80002D0486E0F801A2E8B1E001900D928A9549
:102D9000E1F75FC0C8010E94121A811185CF8091AE
:102DA0008701816080938701C8010E942D0451C072
:102DB00086E0F50111928A95E9F74BC0EE2009F4FF
:102DC00085CFC8010E94121AF82E882309F47ECFFD
:102DD00086E0F801A2E8B1E001900D928A95E1F752
:102DE00080918201909183010E94711592959F704C
:102DF000963051F4863F41F08091810191E089271E
:102E000080938101909380010E94051522C03D8727
:102E10002E878D859E850E947115292F22952F70F2
:102E2000223028F49F7039F0811105C00BC0243086
:102E300028F49F7049F4805E883020F0C8010E9419
:102E40002D049F2CF92C05C0F8019581907F99F7EE
:102E5000F9CF8F2D61960FB6F894DEBF0FBECDBFB0
:102E6000DF91CF911F910F91FF90EF90DF90CF9066
:102E7000BF90AF909F900895CF93DF93CDB7DEB70B
:102E80002A970FB6F894DEBF0FBECDBF84B7877FF9
:102E900084BF0FB6F894A8958091600088618093F4
:102EA0006000109260000FBE90E080E80FB6F894CA
:102EB00080936100909361000FBE85B7806885BFE5
:102EC00085B7806885BF89E491E190934F01809335
:102ED0004E010E94C00F0E94DF0F8091E2008460CB
:102EE0008093E200789480916E018823A1F0109184
:102EF000E9001F709091EC00892F817090FD80E8AF
:102F0000182B1092E9008091E80083FD0E94AF0C1D
:102F10001F701093E90082E084BD93E095BD9AEFA5
:102F200097BD80936E000FE311E037E4E32E31E0AC
:102F3000F32ED8018D918D018F3F11F00E948E11DB
:102F4000E016F106B1F707E411E0F80181918F0175
:102F50008F3F11F00E948E11F1E00D341F07A9F789
:102F600088E0ECEDF1E0DF01282F1D922A95E9F7CA
:102F7000EDECF1E0DF011D928A95E9F7269A2E9A91
:102F8000259A2D9A80E090E00E94761D893E9E4F02
:102F900011F00E940D1482E090E00E946E1D80935B
:102FA000E4010E94FC139093DA018093D90183E03D
:102FB00090E00E946E1D682F70E080E090E00E941B
:102FC000081A3E9A469882E88093900089E180939F
:102FD00091008FEF9FEF90939700809396000E944F
:102FE000401D80910C0281FF0BC010920F021092C5
:102FF0000E0210920D028091710081608093710029
:103000000E94401D81E091E090931602809315028A
:1030100098E1C92ED12C20E4B22EAA24A39480E1F9
:10302000E82E80916E01853009F05BC012E180913D
:103030006E01853009F045C080916E01843009F43D
:103040002FC080910C0280FF04C00E941B1DA09223
:10305000DB0180E00E94E81C80E00E941F041092C7
:1030600019020FB6F894A895C09260000FBEB092F6
:10307000600083B7817F846083BF83B7816083BF33
:103080007894889583B78E7F83BF0FB6F894A89500
:1030900080916000886180936000109260000FBE94
:1030A00080916D01882309F4C2CF0E94A511ECED37
:1030B000F1E08191811174C021E0E43EF207C9F78B
:1030C000B6CF0E94321A0E94401D0E94D31B0E945C
:1030D0001F048091DB01882321F00E94281D10929B
:1030E000DB010E94A511882359F08FB7F894409115
:1030F0005A0150915B0160915C0170915D018FBF3D
:10310000ACEDB1E0E5EEF1E000E010E0302F2D9104
:103110009191922721F180E0FF24F3944F2D4923D0
:10312000D1F089833A832F2181E009F480E08B83F9
:103130000E943D118160782F9D838C8349815A8143
:103140006B818D810E943703F801EB51FE4F808126
:10315000F826F08219C08F5FFF0C8630F9F60F5FFA
:103160001F4F0830110591F68FEF8E838F831886DD
:103170000E943D118160782F9A8789874E815F81F7
:1031800068858A850E9437030E94D31B9091ED01C8
:10319000891709F446CF8093ED010E941F043FCFA9
:1031A000E9BC19BD09B400FEFDCF8091D8008F7D28
:1031B0008093D8008091E00082608093E00080914D
:1031C000E00081FDFCCF0E94321A31CF80E090E018
:1031D0000E94BD1B80E090E00E94A71B1092C301DB
:1031E0000C9485148F929F92AF92BF92DF92EF92D0
:1031F000FF920F931F93CF93DF938090D501909010
:10320000D601A090D701B090D8014091C60150914D
:10321000C7016091C8017091C901842A952AA62A24
:10322000B72ACFE1D0E026E0929F7001112490E30D
:10323000D92E082F10E0D501C4010C2E04C0B6957C
:10324000A795979587950A94D2F780FD04C021979A
:1032500090F780E014C0DC9EF001DD9EF00D11249B
:10326000EE0DFF1DE00FF11FEE0FFF1FEF5BFD4F97
:10327000859194910E946B12019749F38C2FDF91F5
:10328000CF911F910F91FF90EF90DF90BF90AF9083
:103290009F908F900895292F220F920F990F890FD9
:1032A000682F669566956695982F977085E0689F5C
:1032B000B001112440E050E080E0FB01E40FF51F75
:1032C000E251FE4F208130E0092E02C0369527954D
:1032D0000A94E2F721703327042E01C0220F0A94CA
:1032E000EAF7822B4F5F5F4F4530510531F7089564
:1032F000292F220F920F990F890FE82FE695E69557
:10330000E695877051E001C0550F8A95EAF785E090
:10331000E89FF0011124E251FE4F20E030E070E020
:103320004081CB01022E02C0969587950A94E2F760
:103330008170819584278523842781932F5F3F4F58
:103340002530310569F708950F931F938B019C0178
:103350000073112722273327DC01CB01003311052D
:103360002105310511F4806401C08F7B8093D50164
:103370009093D601A093D701B093D8011F910F91DC
:103380000C94E6180F931F9341E050E060E070E06A
:1033900004C0440F551F661F771F8A95D2F74095CA
:1033A0005095609570958091D5019091D601A0912E
:1033B000D701B091D8018A019B01082319232A2340
:1033C0003B23C901B8011F910F910C94A4190F93CD
:1033D0001F9341E050E060E070E004C0440F551FCF
:1033E000661F771F8A95D2F78091D5019091D601FB
:1033F000A091D701B091D8018A019B01082B192B0C
:103400002A2B3B2BC901B8011F910F910C94A419D1
:103410006093C6017093C7018093C8019093C9015E
:103420000C94E618FC01808191810E94711592959F
:103430009F70963079F010F4925001C09A509230FB
:1034400068F4803F69F018F4883E40F409C0843F76
:1034500029F406C0883E20F0813F11F080E00895F5
:1034600081E008951092C40186E0EAE7F1E0DF010F
:103470001D928A95E9F70C94E618882321F00E94A2
:103480007E140C9485140895882339F09091C4011A
:10349000892B8093C4010C9485140895882371F1BD
:1034A0009CEF980F913A60F4E8E7F1E0928189137C
:1034B00001C01282319691E0EE37F907B9F70DC0DD
:1034C00090E2980F983058F4982F977081E001C0DF
:1034D000880F9A95EAF70E947E140C9485149BE558
:1034E000980F933020F480E090E00C94BD1B885A34
:1034F000873120F480E090E00C94A71B0895CF93CF
:10350000882309F453C09CEF980F913AF8F4C82F20
:10351000EAE7F1E080E891E02191C21721F08E17EF
:103520009F07D1F70DC0E8E7F1E08281C81301C021
:103530001282319641E0EE37F407B9F70E94851404
:103540006C2F88E791E00E948D1B13C090E2980FCA
:10355000983090F4877021E030E0A90102C0440F58
:10356000551F8A95E2F7CA019091C401892B809377
:10357000C401CF910C948514EBE5E80FE33040F4DF
:10358000F0E0E25FFE4F808190E0CF910C94BD1B94
:10359000885A873158F4E82FF0E0EE0FFF1FEF5EF6
:1035A000FE4F80819181CF910C94A71BCF910895FC
:1035B0008F929F92AF92BF92CF92DF92EF92FF9243
:1035C0000F931F93CF93DF938C018091960090917E
:1035D00097006CE070E00E94C01D6017710730F02A
:1035E000C80169E070E00E94C01D60C08091960033
:1035F00090919700E0909600F0909700E0919600EF
:10360000F0919700C6E0D0E0BE010E94C01D20E00E
:1036100030E0060F171F211D311D4801590185E0BB
:10362000880C991CAA1CBB1C8A95D1F7C701BE0146
:103630000E94C01D6F01E12CF12CA7019601260FFD
:10364000371F411D511DC501B4010E94D41D6901E0
:103650007A01E0919600F0919700CA01B9010E94A9
:10366000B01D9B01AC01DF010E940B1E9B01AC0150
:10367000C701B6010E94B01DDC01CB012FE0B69559
:10368000A795979587952A95D1F700919600109167
:10369000970020E030E0081719072A073B0728F4B5
:1036A0006091960070919700CB01BC01CB01DF9136
:1036B000CF911F910F91FF90EF90DF90CF90BF902F
:1036C000AF909F908F9008951F920F920FB60F9218
:1036D00011248F939F93AF93BF938091190281110F
:1036E00013C080915A0190915B01A0915C01B0914F
:1036F0005D014196A11DB11D80935A0190935B011C
:10370000A0935C01B0935D01BF91AF919F918F91A8
:103710000F900FBE0F901F9018959C01FC013296E0
:103720009FEF80E04191461789F09F3F19F44111C6
:1037300001C0982F8F5F8630A9F79F3F39F0F901BC
:10374000E90FF11D97FDFA95628308950895209180
:103750001702309118022817390771F09093180258
:1037600080931702E0911502F0911602309721F034
:103770000084F185E02D0994089520911302309181
:1037800014022817390771F09093140280931302E2
:10379000E0911502F0911602309721F00680F78132
:1037A000E02D09940895E0911502F09116023097EA
:1037B00021F00190F081E02D099480E00895EF92CE
:1037C000FF920F93CF93DF93C42FD22FFC018281FE
:1037D0008823D1F0409312020E943D119093110270
:1037E0008093100280E28C0F883008F078C0C77098
:1037F00081E001C0880FCA95EAF7DF91CF910F9160
:10380000FF90EF900C94441A80911202481356C016
:1038100020911002309111024FB7F89480915A0113
:1038200090915B01A0915C01B0915D014FBF821B43
:10383000930B883C910508F041C0CD17C9F080E298
:103840008C0F883040F4C77081E001C0880FCA95A2
:10385000EAF70E943D1A80E28D0F883048F481E03B
:103860009D2F977001C0880F9A95EAF70E94441A1D
:10387000093319F0E12CF12C03C080E5E82EF12C7E
:10388000802F0E947F1AE114F10451F08FE99FE02C
:103890000197F1F700C0000091E0E91AF108F3CFB9
:1038A000802F0E944E1A80E28D0F8830C0F4D770AE
:1038B00081E001C0880FDA95EAF70AC080E28C0F38
:1038C000883068F4C77081E001C0880FCA95EAF7B4
:1038D000DF91CF910F91FF90EF900C943D1ADF9103
:1038E000CF910F91FF90EF9008951F920F920FB616
:1038F0000F9211242F933F934F935F936F937F9376
:103900008F939F93AF93BF93EF93FF9380910D019C
:1039100091E0980F823019F090930D0148C081E03A
:1039200080930D0180910E0290910F02019660ED3F
:1039300072E00E94C01D90930F0280930E0265E01A
:1039400070E00E94C01D6F7780910D02823019F4E3
:10395000603451F404C0813039F46F3729F4809118
:1039600071008E7F80937100E62FF0E0EF5BFA4FDD
:10397000E4912091960030919700E29FC001E39F6F
:10398000900D11246BEF74E00E94C01D80910C0219
:10399000869586958695282F269FC001279F900D96
:1039A00011240E94D81A9093990080939800FF9157
:1039B000EF91BF91AF919F918F917F916F915F91A7
:1039C0004F913F912F910F900FBE0F901F90189520
:1039D000863048F4811108C0909190009F779093B1
:1039E0009000469806C085E0909190009068909372
:1039F0009000A0919600B0919700282F30E00E948F
:103A0000FC1D25E030E040E050E00E94D41DB42FC2
:103A1000A32F922F8827892F9A2FAB2FBB270E9485
:103A2000D81A90939900809398000895682F86E0A3
:103A300090E00C947C1D80910C0280FF08C08E7F6A
:103A400080930C020E94161D80E00C94E81C0895DF
:103A500080910C0280FD13C0816080930C02813044
:103A600019F489E080930C0280910C020E94161DCB
:103A700080910C028695869586950C94E81C089595
:103A800080E090E00E94761D893E9E4F51F00E949A
:103A90000D1480910C028470896280930C020E9444
:103AA000161D86E090E00E946E1D80930C02282F68
:103AB00026952695269530E02630310524F087702E
:103AC000886280930C0280910C0280FF04C086956E
:103AD0008695869501C080E00C94E81CF999FECF8C
:103AE00092BD81BDF89A992780B50895A8E1B0E00C
:103AF00042E050E00C94A21D262FF999FECF92BD12
:103B000081BDF89A019700B4021639F01FBA20BDA2
:103B10000FB6F894FA9AF99A0FBE08950396272FD4
:103B20000E947D1D0E947C1D252F0E947D1D242F3B
:103B30000C947D1D0196272F0E947D1D0C947C1DE9
:103B4000DC01CB01FC01F999FECF06C0F2BDE1BD5D
:103B5000F89A319600B40D9241505040B8F708954C
:103B6000DB018F939F930E940B1EBF91AF91A29F89
:103B7000800D911DA39F900DB29F900D112408956B
:103B8000AA1BBB1B51E107C0AA1FBB1FA617B70783
:103B900010F0A61BB70B881F991F5A95A9F780959F
:103BA0009095BC01CD010895A1E21A2EAA1BBB1B62
:103BB000FD010DC0AA1FBB1FEE1FFF1FA217B307F9
:103BC000E407F50720F0A21BB30BE40BF50B661F0F
:103BD000771F881F991F1A9469F7609570958095D3
:103BE00090959B01AC01BD01CF010895EE0FFF1F21
:103BF0000590F491E02D0994A29FB001B39FC001FC
:103C0000A39F700D811D1124911DB29F700D811D08
:103C10001124911D08950E94FC1DA59F900DB49F35
:103C2000900DA49F800D911D11240895FB01DC01CE
:103C300004C08D910190801921F441505040C8F783
:0A3C4000881B990B0895F894FFCF3C
:103C4A00014D0C830C4C0C7F0C7B0C4B0C018182BC
:103C5A0083E200E900EA00B500B600B700CD0083B0
:103C6A0001CC008A01920194012102230224022537
:103C7A0002260227022A02B300B4006F007000F481
:0E3C8A00F53133919097C6939234F6F73200DD
:00000001FF
